:100000000C9438060C941C240C9470060C94700606
:100010000C9470060C9470060C9470060C94700688
:100020000C9470060C9470060C94FE2C0C94D02D3D
:100030000C9403270C9470060C9470060C947006B4
:100040000C9470060C9470060C9470060C94700658
:100050000C9470060C94A7270C9470060C947006F0
:100060000C9470060C9470060C9470060C94700638
:100070000C9470060C9470060C9470060C94700628
:100080000C9470060C9470060C9470060C94700618
:100090000C9470060C9470060C9470060C94700608
:1000A0000C9470060C9470060C947006A309A309B6
:1000B000CF09CF09370A550A6D0B6D0B600AF90A93
:1000C0000A0B0A0B682156216F21E1201C221C22F9
:1000D00053211C221C229C211C22B021FC211C2209
:1000E0001C221C221C22D0211C221C22CD211C22BD
:1000F00088211C221C2216221622162216221622C3
:10010000162216221622162218221C2268214B21A2
:100110001C221C221C221C221C221C221C221C22EF
:100120001C221C2218221C221C2253211C221422B5
:10013000142214221422142214221422142214220F
:1001400018223D2E642E5C2F642E5C2FB02ED32EF1
:100150005C2F2A2F392F29001E001F0020002100AC
:10016000220000002B0014001A00080015001700E0
:100170000000390004001600070009000A00000012
:10018000E1001D001B000600190005000000E00052
:100190004A0049004C00E3002C00E200000023006C
:1001A00024002500260027002D0000001C00180058
:1001B0000C00120013002E0000000B000D000E00BA
:1001C0000F0033003400000011001000360037002B
:1001D0003800310028002A0001512F0030004D0066
:1001E000350035003A003B003C003D003E00000079
:1001F0000100010001000100005C0100000001009D
:1002000001000100010001000100000001000100E7
:100210000100010001000100000001004B0001008D
:10022000010001000100010000003F00400041000A
:1002300042004300440000000100010052000100A0
:10024000AE00450000000100500051004F00AA0020
:10025000A90000000100A800AC00AB0001000100F3
:10026000010001000100010001004E0001004445B1
:100270004255473A2064697361626C65642E0A00D6
:1002800044454255473A20656E61626C65642E0AAA
:10029000000A0025303258006C65645F7461736B2E
:1002A0003A20004F6E6573686F743A206163746919
:1002B00076653A2025640A000A0025303862003A43
:1002C000200025303258000A722F6320303132333B
:1002D000343536370A0054617267657420636F6E77
:1002E0006E65637465640D0A0054617267657420FD
:1002F000646973636F6E6E65637465642C207468E3
:10030000726F74746C696E6720636F6E6E65637470
:10031000696F6E20617474656D7074730D0A0046A8
:1003200061696C656420746F2065786563757465B8
:100330002025730A00290A002575002F0025750065
:100340005D2800256400200025640020002564004D
:1003500020002564007C0025303258006D6F7573D5
:10036000656B6579205B62746E7C782079207620DD
:10037000685D287265702F61636C293A205B0031DB
:100380003A0964656C6179282A31306D73293A2005
:1003900025750A323A09696E74657276616C286D4A
:1003A00073293A2025750A333A096D61785F7370B5
:1003B0006565643A2025750A343A0974696D655F8C
:1003C000746F5F6D61783A2025750A353A09776850
:1003D00065656C5F6D61785F73706565643A202553
:1003E000750A363A09776865656C5F74696D655F93
:1003F000746F5F6D61783A2025750A00703A097054
:1004000072696E742076616C7565730A643A09735B
:1004100065742064656661756C74730A75703A0959
:100420002B310A646E3A092D310A6C743A092B316A
:10043000300A72743A092D31300A4553432F713A0C
:1004400009717569740A0A7370656564203D2064DA
:10045000656C7461202A206D61785F7370656564D6
:10046000202A2028726570656174202F2074696DC0
:10047000655F746F5F6D6178290A776865726520C2
:1004800064656C74613A20637572736F723D2564A4
:100490002C20776865656C3D25640A536565206886
:1004A0007474703A2F2F656E2E77696B697065646E
:1004B00069612E6F72672F77696B692F4D6F757346
:1004C000655F6B6579730A004D3E20004D25753AD6
:1004D00025733E20003F0A003D2025750A003F0A93
:1004E0000064656661756C74730A0025750A003FC7
:1004F0000A000A092D2056616C756573202D0A00CB
:10050000710A000A092D204D6F7573656B6579209E
:100510002D0A003F00433E20004C25640A000A09D2
:100520002D20537461747573202D0A686F73745F86
:100530006B6579626F6172645F6C65647328293AD8
:1005400020253032580A6B6579626F6172645F7082
:10055000726F746F636F6C3A20253032580A6B6586
:1005600079626F6172645F69646C653A202530322C
:10057000580A6B65796D61705F636F6E6669672E8F
:100580006E6B726F3A20253032580A74696D65724D
:100590005F72656164333228293A202530386C58FF
:1005A0000A000A092D2056657273696F6E202D0AA4
:1005B0005649443A2030784645454428426C616E9D
:1005C0006B205465686E6F6C6F67696929205049AC
:1005D000443A20307830303030284D616E69627591
:1005E0007329205645523A203078303030320A4252
:1005F00055494C443A202028466562203237203243
:10060000303232290A4F5054494F4E533A204C55FC
:100610004641204D4F5553454B455920455854525E
:10062000414B455920434F4E534F4C4520434F4D6E
:100630004D414E44204E4B524F20343039360A47FC
:1006400043433A20352E342E30204156522D4C490A
:1006500042433A20322E302E30204156525F4152D2
:1006600043483A20617672350A000A092D20436F0B
:100670006E736F6C65202D0A4553432F713A0971D3
:100680007569740A6D3A096D6F7573656B65790AE2
:10069000000A092D204D61676963202D0A443A093B
:1006A0004465627567204D65737361676520546F9B
:1006B00067676C650A583A094D617472697820441D
:1006C00065627567204D6F646520546F67676C6560
:1006D000202D2053686F77206B6579707265737376
:1006E000657320696E206D61747269782067726924
:1006F000640A4B3A094B6579626F61726420446504
:1007000062756720546F67676C65202D2053686F92
:1007100077206B65797072657373207265706F7284
:10072000740A4D3A094465627567204D6F757365AB
:1007300020546F67676C650A563A0956657273698B
:100740006F6E0A533A095374617475730A433A0918
:10075000416374697661746520436F6E736F6C6575
:10076000204D6F64650A46312D4631303A09537782
:100770006974636820746F204C6179657220302D34
:10078000392028463130203D204C30290A302D397F
:100790003A0953776974636820746F204C617965F6
:1007A0007220302D390A47524156453A095377692C
:1007B00074636820746F204C617965722030202842
:1007C000616C7465726E617465290A423A094A75F2
:1007D0006D7020746F20426F6F746C6F616465720E
:1007E0000A4553433A094A756D7020746F20426F71
:1007F0006F746C6F616465722028616C7465726ED1
:10080000617465290A453A095072696E742045453C
:1008100050524F4D2053657474696E67730A42538A
:10082000504143453A09436C656172204545505239
:100830004F4D0A4E3A094E4B524F20546F67676C2A
:10084000650A006B65796D61705F636F6E666967DD
:100850002E7261773A20253032580A2E73776170F4
:100860005F636F6E74726F6C5F636170736C6F63E4
:100870006B3A2025750A2E636170736C6F636B5F32
:10088000746F5F636F6E74726F6C3A2025750A2EF9
:10089000737761705F6C63746C5F6C6775693A2025
:1008A00025750A2E737761705F7263746C5F72676F
:1008B00075693A2025750A2E737761705F6C616CDB
:1008C000745F6C6775693A2025750A2E73776170BD
:1008D0005F72616C745F726775693A2025750A2EC4
:1008E0006E6F5F6775693A2025750A2E73776170A0
:1008F0005F67726176655F6573633A2025750A2EBE
:10090000737761705F6261636B736C6173685F6260
:1009100061636B73706163653A2025750A2E6E6B97
:10092000726F3A2025750A0064656275675F636FB0
:100930006E6669672E7261773A20253032580A2E2A
:10094000656E61626C653A2025750A2E6D61747260
:1009500069783A2025750A2E6B6579626F61726439
:100960003A2025750A2E6D6F7573653A2025750A34
:10097000006565636F6E6669673A0A6465666175EE
:100980006C745F6C617965723A2025750A003F00CE
:100990004E4B524F3A206F66660A004E4B524F3A0A
:1009A000206F6E0A000A6D6F7573653A206F666678
:1009B0000A000A6D6F7573653A206F6E0A000A6B44
:1009C0006579626F6172643A206F66660A000A6B2D
:1009D0006579626F6172643A206F6E0A000A6D6118
:1009E000747269783A206F66660A000A6D617472E3
:1009F00069783A206F6E0A000A64656275673A206A
:100A00006F66660A000A64656275673A206F6E0A4F
:100A1000000A0A4A756D70696E6720746F20626FF4
:100A20006F746C6F616465722E2E2E2000433E2021
:100A300000436C656172696E6720454550524F4DA9
:100A40000A000A002530325820006B6579626F6118
:100A500072645F7265706F72743A200064656C5FD7
:100A60006B65795F6269743A2063616E27742064F4
:100A7000656C3A20253032580A006164645F6B650A
:100A8000795F6269743A2063616E277420616464DF
:100A90003A20253032580A005B735D005B575D00D9
:100AA0005B535D005B525D005B445D005B435D003A
:100AB00010034D0061006E00690062007500730054
:100AC0000000220342006C0061006E006B002000F9
:100AD0005400650068006E006F006C006F006700D6
:100AE0006900690000000403090409025B000301B6
:100AF00000A0FA090400000103010100092111010D
:100B000000012240000705810308000109040100DB
:100B1000010300000009211101000122B6000705B0
:100B200082032000010904020002030000000921E1
:100B3000110100012222000705830320000107059F
:100B400003032000011201000200000008EDFE0076
:100B5000000200010200010631FF0974A1010975BC
:100B6000150026FF009520750881020976150026DC
:100B7000FF00952075089102C005010902A10185B9
:100B8000020901A10005091901290815002501958F
:100B900008750181020501093009311581257F950C
:100BA000027508810609381581257F950175088130
:100BB00006050C0A38021581257F95017508810606
:100BC000C0C005010980A101850319012AB70015DC
:100BD0000126B700950175108100C0050C0901A11F
:100BE00001850419012AA002150126A002950175AC
:100BF000108100C005010906A1018506050719E05D
:100C000029E71500250195087501810205071900DE
:100C100029EF1500250195F07501810205081901DC
:100C20002905950575019102950175039101C0058E
:100C3000010906A101050719E029E715002501951D
:100C400008750181029501750881010507190029C0
:100C5000FF150026FF00950675088100050819019B
:100C60002905950575019102950175039101C00053
:100C700011241FBECFEFDAE0DEBFCDBF04B603FE06
:100C800018C08091920390919303A0919403B09126
:100C900095038730904BA740B04B59F410929203C4
:100CA000109293031092940310929503E0E0F8E3FE
:100CB000099512E0A0E0B1E0EAE6F0E602C0059096
:100CC0000D92A233B107D9F723E0A2E3B2E001C04D
:100CD0001D92A239B207E1F70E94F21A0C94333048
:100CE0000C940000FF93EF93E0913202F0913302F5
:100CF000309709F00995EF91FF910895FC018591D6
:100D0000803011F0EFDFFBCF0895FF27E0E230E203
:100D100047FF0CC0419597FF09C0EDE260957095C3
:100D200080959095611D711D811D911D27FF02C049
:100D3000219530E350E2AA27660F771F881F991F7D
:100D4000AA1FA41710F0A41B63955A95A9F7AA30FF
:100D500008F0A95FA05DAF93F3956115710581055A
:100D6000910541F7ED3211F4EF93F395F21718F472
:100D70003F93F395FBCF8F91B5DFFA95E1F7089597
:100D8000E991F9918591803021F0853219F0AADF3F
:100D9000F9CF089520E0E89455915532C1F35033CE
:100DA00011F4689455915A3348F4505390F3220F3C
:100DB000022E220F220F200D250FF4CF0EF42195C5
:100DC00089919991533619F3533729F1533559F1D4
:100DD000BC0188279927E8945C3621F48991999180
:100DE00068945591543639F446EF7EF077FF0DC084
:100DF0008FEF9FEF0AC055374AE039F0583540E190
:100E000021F0523642E009F00895FF93EF937DDF21
:100E1000EF91FF91B7CFFF93EF93FC018191803069
:100E2000B9F360DFFBCFFF93EF9368DFF1CFDF9380
:100E3000CF93CDB7DEB72596A3DFCF91DF9108958D
:100E400081E0089581E008950C94220708950C94A0
:100E500026071F93CF93DF9300D000D01F92CDB70A
:100E6000DEB749835A836B833091350289819A8139
:100E7000311114C0662359F0222349F00E94AA0DB3
:100E8000182F682F89819A810E94530D03C00E94F8
:100E90007E0D182F69817A81812F04C00E94AA0DCE
:100EA00069817A810F900F900F900F900F90DF91D2
:100EB000CF911F910C94EB14FC01262F408151819E
:100EC0006281738184810C94290781E00895CF9316
:100ED000DF93EC0160E00E945C07BE01DF91CF91DF
:100EE0000C9427070C949B160C94971608950E9457
:100EF000FD0B0E9476072FEF84E39CE02150804099
:100F00009040E1F700C000000C94CD270F931F9391
:100F1000CF93DF938C0161E00E945C07EC01B80184
:100F20000E942407882309F45BC0B801CE010E9407
:100F30002923882309F454C0B801CE010E94221E3F
:100F4000882309F44DC0B801CE010E948522882370
:100F500009F446C0F80182818823D9F1CF3D8CE5A0
:100F6000D80779F140F4C115FCE5DF0791F0C130F5
:100F7000DC4591F02EC0CC35EDE5DE0741F1CD35F5
:100F8000FDE5DF0709F1CB35DD4519F50E9441127A
:100F900020C00E94770724C08091F902C82FC09515
:100FA000C170C0FB80F98093F902CC2329F080E85E
:100FB00092E00E947E0614C08EE692E00E947E06B9
:100FC00010C00E94EF120CC00E94381202C00E9492
:100FD0004412C801DF91CF911F910F910C9420070B
:100FE000C0E08C2FDF91CF911F910F9108950E9447
:100FF000E6260C9422080E9425080C94EC26829583
:10100000982F937344E0949F900111248C7C8695D3
:101010008695282B822F8575880F2A7A2695822B14
:10102000089508950C94110881E008950C94140813
:101030000895CF93C82F0E9412088C2F0E94160883
:10104000CF91089580E00C9419080E9447250C94D4
:101050001908CF930E944725C82F80913402C817E2
:1010600041F1C09334028091F90282FF1EC080FFDB
:1010700004C088E992E00E947E068091F90280FF18
:101080000CC01F92CF9383E992E09F938F930E94AD
:1010900017070F900F900F900F908091F90280FF2B
:1010A00004C081E992E00E947E068C2FCF910C94BF
:1010B0001908CF910895CF93DF93CDB7DEB72B9763
:1010C0000FB6F894DEBF0FBECDBF4F835887698738
:1010D0007A878B8761110E9470119E012F5F3F4FAD
:1010E00086E0F90111928A95E9F785E0FE013796CD
:1010F000D90101900D928A95E1F789819A814C81FD
:101100005D81452B31F09F3F31F491E08F3F19F421
:1011100003C091E001C090E090FF09C049815A816D
:101120006B817C818D819E810E94911005C0C901D7
:101130000E9465078111F2CF2B960FB6F894DEBF9F
:101140000FBECDBFDF91CF910895FC0180819181C9
:101150000E94EC0D0895CF93882309F455C0C82F41
:101160008CEF8C0F813AF8F48C2F0E942E22811183
:101170004BC06C2F80910201909103010E94FF25CA
:10118000882349F06C2F80910201909103010E9405
:10119000AC260E9492116C2F809102019091030164
:1011A0000E94A1260CC080E28C0F883058F4C770D2
:1011B00081E001C0880FCA95EAF70E945311CF91D0
:1011C0000C949211EBE5EC0FE33040F4F0E0E858BA
:1011D000FE4F808190E0CF910C94BD25E8E5EC0FA7
:1011E000E73150F4F0E0EE0FFF1FE65BFE4F808129
:1011F0009181CF910C94D325CD3E30F08C2F0E945D
:10120000771BCF910C94491CCF910895882389F1C5
:101210009CEF980F913A40F4682F809102019091D1
:1012200003010E94AC260DC090E2980F983058F44C
:10123000877091E001C0990F8A95EAF7892F0E9483
:1012400059110C9492119BE5980F933020F480E093
:1012500090E00C94BD2598E5980F973120F480E03C
:1012600090E00C94D3258D3E20F00E94D21B0C946C
:10127000491C08951F93CF93DF93182FEB010E9411
:10128000AB08209741F08FE99FE00197F1F700C08C
:1012900000002197F6CF812FDF91CF911F910C9401
:1012A0000609893319F060E070E002C060E570E083
:1012B0000C943A09882321F00E9453110C94921146
:1012C0000895882321F00E9459110C9492110895D9
:1012D000CF92DF92EF92FF920F931F93CF93DF9302
:1012E0007C01D62FC72FFC011281058102950F705A
:1012F0000E9449118823B9F01123A9F08C2F807F17
:10130000803421F080E28D0F883068F080916A038C
:1013100082FD09C082E00E94F2110E94491191E011
:10132000D82ED92601C0D12CCC2EC2948FE0C82251
:101330008C2D90E08C30910508F0CFC1FC01EA5A69
:10134000FF4F0C94C12F8C2F807FCF70882311F01A
:10135000C295C07F112399F0CC2309F4AAC180E281
:101360008D0F883010F0D11104C08C2F0E945311C2
:1013700003C08C2F0E9463110E9492119AC18D2F7D
:101380000E940609CC2309F4A8C180E28D0F8830A1
:1013900038F1DD2329F18C2F0E94691124C08C2F94
:1013A000807FCF70803211F0C295C07FDD2319F0AD
:1013B000D130A1F13DC080916A0382FF17C0112393
:1013C00049F0CC2329F08C2F0E9453110E949211D6
:1013D00080E070C180E00E940609CC2309F47DC141
:1013E0008C2F0E9459110E94921177C1112371F024
:1013F000002341F0013031F40E9473118C2B0E94C4
:101400007B116BC10E9473118C2B1DC0002319F03E
:10141000013009F462C10E94881125C0112321F016
:10142000063008F05AC10EC0053008F056C11BC086
:10143000112361F0002331F0F701858180FF39C16C
:101440008F7085838C2F0E945A0947C1002359F061
:10145000D93309F03FC1FFEF07EE13E0F150004030
:101460001040E1F735C18C2F0E94610936C18C2FE5
:1014700086958695837019F0813061F02EC1112315
:1014800021F08D2F9C2F937002C080E090E00E948D
:10149000BD252BC1112321F08D2F9C2F937002C0ED
:1014A00080E090E00E94D32520C18D2F112319F0F8
:1014B0000E94771B02C00E94D21B0E94491C15C1CA
:1014C0008C2F837009F047C011110BC12D2F22956D
:1014D00026952770220F220F6D2F6F70862F90E0B8
:1014E000A0E0B0E0022E04C0880F991FAA1FBB1F06
:1014F0000A94D2F7D4FF10C04FE050E060E070E0F3
:1015000004C0440F551F661F771F2A95D2F74095D8
:1015100050956095709503C040E050E0BA01C695C3
:10152000C695C3708A019B01082B192B2A2B3B2BD4
:10153000C901B801C23049F058F4C13019F00E9415
:10154000690CCFC00E94570CCCC00E947B0CC9C054
:101550000E94550CC6C0112319F08C2F817001C058
:101560008695882309F4BDC02D2F229526952770D6
:10157000220F220F6D2F6F70862F90E0A0E0B0E059
:10158000022E04C0880F991FAA1FBB1F0A94D2F70E
:10159000D4FF10C04FE050E060E070E004C0440FA2
:1015A000551F661F771F2A95D2F740955095609575
:1015B000709503C040E050E0BA01C695C695C3706F
:1015C0008A019B01082B192B2A2B3B2BC901B8013F
:1015D000C23049F058F4C13019F00E942E0D81C07C
:1015E0000E941C0D7EC00E94400D7BC00E948F0C8B
:1015F00078C0CF70112339F08C2F0E94B50C8D2F3D
:101600000E945A096EC08D2F0E9461098C2F0E9482
:10161000D60C67C0D23F21F128F4D03F41F0D13F32
:10162000C1F043C0D33F19F1D43F79F03EC011233C
:1016300041F0053008F051C08C2F8F710E94FB0CD7
:101640004CC0063008F049C0F7CF80916A0382FF92
:1016500018C0112339F08C2F8F710E94B50C3DC03A
:101660001123C9F38C2F8F710E94D60C36C0112321
:1016700029F08C2F8F710E94A00C2FC00E949B0C10
:101680002CC0112349F0CF718C2F0E94B50C63E060
:101690008C2F0E94D71121C081E00E94F2110230EC
:1016A000E0F082E00E94F21118C0112331F0002313
:1016B00091F28D2F0E94AB0810C0002399F2D9330C
:1016C00049F41FEF27EE33E0115020403040E1F79E
:1016D00000C000008D2F0E94060988EF8C0D843019
:1016E00020F40E9447250E941908DD20C9F00E94BD
:1016F000451180FD15C0F70112820E943F110E9422
:10170000B50CC7010E94B10B0E943F11DF91CF9130
:101710001F910F91FF90EF90DF90CF900C94D60C1B
:10172000DF91CF911F910F91FF90EF90DF90CF90BD
:1017300008950F931F93CF93DF93EC016881798114
:101740008A810E94F70D8C010E94520D0E94430C69
:10175000B801CE010E946809DF91CF911F910F91CE
:101760000895CF93DF93EC01988189812B813C818F
:10177000232B31F08F3F31F481E09F3F19F403C0F8
:1017800081E001C080E080FD1DC0CE010E9486077F
:10179000811110C00E9449118823A1F08A818823F9
:1017A00089F080916A0382FD0DC082E0DF91CF91C4
:1017B0000C94F211CE010E94990BCE01DF91CF91D2
:1017C0000C946707DF91CF91089580E090E00E942C
:1017D000BD2580E090E00E94D3250E9470110E94F8
:1017E00092110E94FC1D0C94491C80910201909161
:1017F00003010E94B7260C94E50B0E9460110C9423
:10180000F50B92959F70963079F010F4925001C0CC
:101810009A50923068F4803F69F018F4883E40F4A2
:1018200009C0843F29F406C0883E20F0813F11F0B2
:1018300080E0089581E00895FC01808191810E94FB
:10184000EC0D0E94010C0895CF93DF9300D000D0DF
:101850001F92CDB7DEB70F900F900F900F900F90A3
:10186000DF91CF910895CF93DF9300D000D000D0C7
:10187000CDB7DEB726960FB6F894DEBF0FBECDBF4C
:10188000DF91CF910895089508950C94440C0C9421
:10189000450C0E94470C6093670270936802809326
:1018A000690290936A020C94E50B0C94490C0F9317
:1018B0001F93009167021091680220916902309194
:1018C0006A02602B712B822B932B1F910F910C942A
:1018D000490C0F931F9300916702109168022091A9
:1018E000690230916A0260237123822393231F913E
:1018F0000F910C94490C0F931F9300916702109164
:1019000068022091690230916A026027712782275C
:1019100093271F910F910C94490C0C94440C0E9436
:101920008D0C6093630270936402809365029093C0
:1019300066020C94E50B60E070E0CB010C948F0C18
:101940000F931F9341E050E060E070E08A019B013B
:1019500004C0000F111F221F331F8A95D2F7C9013F
:10196000B8011F910F910C948F0C0F931F9341E0BE
:1019700050E060E070E004C0440F551F661F771F01
:101980008A95D2F78091630290916402A0916502DA
:10199000B09166028A019B01082B192B2A2B3B2B45
:1019A000C901B8011F910F910C948F0C0F931F93D5
:1019B00041E050E060E070E004C0440F551F661F36
:1019C000771F8A95D2F740955095609570958091D4
:1019D000630290916402A0916502B09166028A014F
:1019E0009B01082319232A233B23C901B8011F9116
:1019F0000F910C948F0C0F931F9341E050E060E027
:101A000070E004C0440F551F661F771F8A95D2F7F8
:101A10008091630290916402A0916502B091660288
:101A20008A019B01082719272A273B27C901B801EA
:101A30001F910F910C948F0C0F931F9300916302D1
:101A4000109164022091650230916602602B712B27
:101A5000822B932B1F910F910C948F0C0F931F933C
:101A60000091630210916402209165023091660238
:101A700060237123822393231F910F910C948F0C69
:101A80000F931F93009163021091640220916502ED
:101A90003091660260277127822793271F910F914B
:101AA0000C948F0C089527E0929F800D1124E82F4D
:101AB000E695E695E695877051E001C0550F8A9549
:101AC000EAF785E0E89FF0011124EA5CFD4F20E091
:101AD00030E070E04081CB01022E02C096958795E0
:101AE0000A94E2F781708195842785238427819366
:101AF0002F5F3F4F2530310569F7089527E0929F0A
:101B0000800D1124682F669566956695982F9770BD
:101B100085E0689FB001112440E050E080E0FB01C7
:101B2000E40FF51FEA5CFD4F208130E0092E02C072
:101B3000369527950A94E2F721703327042E01C0C9
:101B4000220F0A94EAF7822B4F5F5F4F4530510511
:101B500031F70895BF92CF92DF92EF92FF920F93E9
:101B60001F93CF93DF938C01C0906302D0906402E7
:101B7000E0906502F09066028091670290916802A1
:101B8000A0916902B0916A02C82AD92AEA2AFB2ADE
:101B9000CFE1D0E0D701C6010C2E04C0B695A795C1
:101BA000979587950A94D2F780FD04C0219790F706
:101BB000B12C07C0BC2EB8018C2F0E94FE140197D7
:101BC000A9F38B2DDF91CF911F910F91FF90EF9093
:101BD000DF90CF90BF900895CF93DF93EC010E94E8
:101BE000AA0DBE010E94FE14DF91CF9108951F93AC
:101BF000CF93DF93EB0190913502992321F0CB0134
:101C00000E94EC0D13C0882349F0CB010E94AA0D5D
:101C1000182F682FCE010E94530D04C0CB010E94E3
:101C20007E0D182FBE01812F0E94FE14DF91CF91EF
:101C30001F9108951F93CF93DF93C0916B0216E01D
:101C400080916C02C81799F0D0E01C9FF0011D9F95
:101C5000F00D1124E359FD4F408151816281738160
:101C6000848195810E94330C2196C770E9CFDF9162
:101C7000CF911F91089540919D0250919E026091D5
:101C80009F027091A0028091A1029091A2020C94F7
:101C9000330CEF92FF920F931F93CF93DF938091BA
:101CA000A20282958F7009F065C080919F028823FF
:101CB00009F460C080916B02F0906C0210919D025B
:101CC00000919E026091A0027091A10291E01F3FDD
:101CD00009F090E0C0910001D0910101292F96E018
:101CE000E92E8F1509F446C06115710521F00F3FEB
:101CF00021F030E003C031E001C0322F90E030FD30
:101D000036C0E89EF001E99EF00D1124DF01A359D1
:101D1000BD4F11963C911197301329C03C9131135E
:101D200026C012963C911297311121C013964D9105
:101D30005C911497461B570B4C175D07C0F48091BC
:101D4000A2028F7080618093A202EE58FD4F8081C5
:101D50008F70806180838DE992E00E94B10BDF91EA
:101D6000CF911F910F91FF90EF900C941A0E019656
:101D70008770B7CFDF91CF911F910F91FF90EF90B8
:101D800008959F92AF92BF92CF92DF92EF92FF920F
:101D90000F931F93CF93DF93CDB7DEB761970FB645
:101DA000F894DEBF0FBECDBF8C0185E0F801DE01E7
:101DB0001D9601900D928A95E1F7D8011296EC904C
:101DC00090919D02E0919E022091A0023091A1028B
:101DD0002115310531F0EF3F31F481E09F3F19F4D7
:101DE00003C081E001C080E0B82FB1709B2E80FD60
:101DF00047C1D8014C9111965C9111971396AD9003
:101E0000BC9014978DE9C82E82E0D82EF0909F02E6
:101E1000B501621B730B2091000130910101FF207D
:101E200009F4D9C08091A2026217730708F095C027
:101E3000282F207F09F052C05E1313C0491311C030
:101E4000FE2CE1100EC08F7080618093A2020E9470
:101E50003B0EC6010E94B10B8091A202F80185835E
:101E60004DC1AB2831F05F3F31F481E04F3F19F4B1
:101E700003C081E001C080E080FD03C081E08E25C9
:101E800002C080E090E0F82FF170FF2E80FF1CC0B0
:101E900080916B0220916C0236E0821709F40BC12D
:101EA00090E0389FF001399FF00D1124E359FD4F68
:101EB0006181561306C06081461303C06281E61239
:101EC00003C001968770E9CFFE2CEE2009F416C1FD
:101ED0008091A20281608093A20254C05E1306C06A
:101EE000491304C0E11002C0F80199C0C8010E9462
:101EF0001C0C882361F1EE2051F12091A202822F67
:101F000082958F7090E0029774F080919D0290917D
:101F10009E0298878F831986BB86AA862C87CE015E
:101F200007960E94B10B86E0F801ADE9B2E001909E
:101F30000D928A95E1F70E94490E0E943B0E0AC05D
:101F40005E1711F1C8010E941C0C81112CC0C80140
:101F50000E94B10BFF24F394D1C0282F207F81F77A
:101F60007A2DB98AA88A6E2D89890E94240C8DE960
:101F700092E00E94B10B86E0D6011D928A95E9F7A6
:101F80000E943B0EF12CBAC04913DCCFE110DACF2E
:101F9000F8018583C8010E94B10B86E0D6011D922D
:101FA0008A95E9F7ABC0EE2091F22091A202822F30
:101FB00082958F7090E002970CF4B5CF80919D02CE
:101FC00090919E029A8389831B82BD82AC822E836C
:101FD000CE010196A6CF6217730708F044C0FE2C0D
:101FE000EE2009F4B4CF5E1330C049132EC0209107
:101FF000A20220FD21C0822F82958F70482F50E0D1
:1020000041155105C9F0F80125834F30510541F0C4
:102010008F5F982F9295907F822F8F70892B858369
:10202000C8010E94B10B86E0F801ADE9B2E0019071
:102030000D928A95E1F73CC086E0F801ADE9B2E087
:1020400001900D928A95E1F759C0C8010E941C0CBD
:10205000811169CF8091A20281608093A202C801A0
:102060000E94B10B4BC07A2DB98AA88A6E2D89893E
:102070000E94240C86E0D6011D928A95E9F718C0CB
:10208000EE2009F464CFC8010E941C0CF82E8823AE
:1020900009F45DCF86E0F801ADE9B2E001900D9260
:1020A0008A95E1F78DE992E00E94A5080E94490E09
:1020B0000E943B0E23C04D875E878D859E850E94C2
:1020C000EC0D292F22952F70223028F49F7039F0C3
:1020D000811105C00BC0243028F49F7049F4805E44
:1020E000883020F0C8010E94B10B9F2CF92C06C04B
:1020F000D80115969C91907F91F7F8CF8F2D61961E
:102100000FB6F894DEBF0FBECDBFDF91CF911F9108
:102110000F91FF90EF90DF90CF90BF90AF909F9086
:1021200008951F93CF93DF93CDB7DEB72C970FB6EB
:10213000F894DEBF0FBECDBF4F83588769877A877B
:102140008B879C87CE0107960E94C10E8823D1F011
:102150009F8188852A853B85232B31F08F3F31F481
:1021600081E09F3F19F403C081E001C080E080FD61
:1021700047C04F81588569857A858B859C850E94EB
:10218000330C3EC086E0FE013796DE0111960190C9
:102190000D928A95E1F7FF81E8856A857B85611557
:1021A000710531F0EF3F31F481E0FF3F19F403C0D6
:1021B00081E001C080E080FD23C020916C0230E00E
:1021C000C90101968770992740916B0250E08417EE
:1021D0009507F1F1F983EA837D836C8396E0929F02
:1021E000D001939FB00D1124A359BD4FFE0131962C
:1021F00001900D929A95E1F780936C020E941A0E5D
:1022000016E080916B0290916C02891771F1189F12
:10221000C001112483599D4F0E94C10E882329F1CA
:10222000E0916B021E9FF0011124E359FD4F4081A4
:10223000518162817381848195810E94330C8091E8
:102240006B0290E001968770992780936B02D9CF3B
:102250000E94FD0B10926C0210926B02EDE9F2E00D
:1022600086E0DF011D928A95E9F72C960FB6F89467
:10227000DEBF0FBECDBFDF91CF911F91089580913A
:10228000C30285958595859508958091C3028770D1
:1022900008959091C302977081E009F480E0089559
:1022A0008091E60208959091E602892B8093E602E0
:1022B000089580959091E60289238093E60208951F
:1022C0001092E60208959091E502892B8093E50231
:1022D000089580959091E50289238093E502089501
:1022E0001092E50208958091C402089508950C9417
:1022F00076110C94771190916A0392FD08C0909129
:10230000C402981721F08093C4020C9479110895A7
:102310008091C402882329F01092C40280E00C94BA
:1023200079110895CF93DF93E0910201F0910301B9
:102330008091E6028083E0910201F0910301908197
:102340008091E502892B80838091C402882381F0EB
:10235000E0910201F09103019081892B80838091AB
:102360000201909103010E94E92581110E948811C8
:10237000C0910201D091030140E250E063EA72E0B3
:10238000CE010E94DB2F892B69F080E2FE01A3EAD7
:10239000B2E001900D928A95E1F7CE01DF91CF91E5
:1023A0000C945A25DF91CF9108950C947611909159
:1023B0006A0392FD10C098E0899F90011124262B9A
:1023C0002093C3020E94B50C8091C3028595859528
:1023D00085950C94D5110C94B50C1092C30280E035
:1023E0000C94D5112091C302809582238093C3025F
:1023F000982F977099F430E0482F082E000C550B59
:102400002417350759F090916A0392FD07C085950E
:10241000859585950E94D60C0C94ED110895CF9367
:1024200090916A0392FB222720F92817F9F0C82F10
:10243000892FC0FB82F980936A0380916903909190
:102440006A030E946B1282E00E94F2118091F902ED
:1024500080FF0CC01F92CF9383EA92E09F938F93EB
:102460000E9417070F900F900F900F90CF91089533
:1024700080916A0382FB882780F991E089270C9478
:102480000F1281E00C940F1280E00C940F1280E088
:1024900090E00E94F92F21E0893E9E4F09F020E054
:1024A000822F089582E090E00C94F12F83E090E079
:1024B0000C94F12FCF9384E090E00E94F12FC82F6D
:1024C00082E290E00E94F12F2C2F30E0A901582BDE
:1024D000CA01CF910895CF93C92F682F84E090E06F
:1024E0000E94FF2F6C2F82E290E0CF910C94FF2F7F
:1024F000AB01BC018FE090E00C941130AB01BC014A
:1025000083E190E00C94113060E070E0CB010C941A
:102510007E1260E070E0CB010E9478120C9484126D
:1025200069EE7EEF80E090E00E941D3060E082E086
:1025300090E00E94FF2F60E083E090E00E94FF2F78
:1025400010926702109268021092690210926A0259
:1025500060E084E090E00E94FF2F60E082E290E083
:102560000E94FF2F60E085E090E00E94FF2F60E076
:1025700086E090E00E94FF2F6FEF87E090E00E94DE
:10258000FF2F40E050E0BA0188E090E00E94113057
:1025900060E08DE090E00E94FF2F40E050E0BA0143
:1025A00088E190E00E94113060E087E190E00E94B5
:1025B000FF2F40E050E0BA018CE190E00E94113022
:1025C00060E070E080E290E00E941D3040E050E06A
:1025D000BA0188E190E00E9411300C9489120C94A9
:1025E00090128EE090E00E94F12F91E0811101C0E5
:1025F00090E0892F0895682F8EE090E00C94FF2FD3
:102600000E9470276093F5027093F6028093F702A0
:102610009093F8026093F1027093F2028093F302B8
:102620009093F402089585B7806885BF85B7806868
:1026300085BF08950C948C1808950C941C130C9469
:102640001C130C941F130C941C130C9423130C9444
:102650001C130E94131389ED99E20E943D250E94EC
:1026600027130C9425130E941D130C941C130E9415
:102670001C160C9418080E945B270E94DA150E9411
:10268000A4180E94A0170E9437130E940A1E0E94DD
:10269000AE180C9421138F929F92AF92BF92CF925B
:1026A000DF92EF92FF920F931F93CF93DF93CDB7FB
:1026B000DEB72A970FB6F894DEBF0FBECDBF0E94DB
:1026C000FF17982E81110E94001387EEA82E82E03A
:1026D000B82E00E010E0802E802F0E944016D82EE9
:1026E000F501C1905F01C826B1F40F5F1F4F0A309A
:1026F000110589F78FEF89838A831B820E946427E3
:102700008160782F9D838C8349815A816B818D8173
:102710000E945B082FC08091F90281FD0E9446163D
:10272000E12CFF24F3948C2D8F21F1F00E941A13D9
:10273000882399F0EE828F82DF2081E009F480E027
:1027400088870E9464278160782F9A8789874E81C5
:102750005F8168858A850E945B08F801E951FD4F19
:102760008081F826F08206C0E394FF0CF7E0EF12B8
:10277000DACFBBCF81E0911001C080E02A960FB67E
:10278000F894DEBF0FBECDBFDF91CF911F910F91A7
:10279000FF90EF90DF90CF90BF90AF909F908F9081
:1027A00008950E944B130E948C180E94E91C0C94FF
:1027B0002908CF93DF930E940315EC01811521E5D1
:1027C000920708F045C0811530E5930708F094C0E2
:1027D000883E910528F5803E910508F0F8C0883ABA
:1027E000910570F4853A910508F07CC0813091051F
:1027F00009F475C008F4E8C0049708F0E8C0E4C024
:102800008F3B910508F0E0C0C85AD0E0CC0FDD1F27
:10281000C558DE4F0990D881C02DCE019464D8C030
:10282000811540E2940758F4811551E0950708F0AE
:10283000CEC08D3E910508F4C7C09065C9C0C115D2
:1028400080E4D80708F4C0C0DF70CE01906AC0C031
:10285000811525E59207A8F4811534E5930708F062
:1028600095C0811543E5940708F07BC0811552E5BA
:10287000950708F061C0D82FCC27CE01816F906AF0
:10288000A7C0C11589E5D807A0F4C11528E5D2076E
:1028900008F082C0C11536E5D30708F095C08C2F2B
:1028A0000E9497158F7190E0D82FCC27CE019062AF
:1028B0008FC0C1154AE5D40708F474C0CE01905604
:1028C0008115904208F080C08D2F8F710E9497155E
:1028D000DD27D0628F71AE01582BCA0179C081E02B
:1028E00090E076C0C55AD0E0C755DE4F8881C82F2A
:1028F000D0E0CE0190646CC074E0969587957A958F
:10290000E1F7282F23703C2F337081E090E002C064
:10291000880F991F3A95E2F79C68AC01522B9A01F7
:102920009C2F9F709695969550E2959FE0011124FB
:10293000C9018C2B9D2B4CC08370992721E030E07E
:1029400002C0220F331F8A95E2F79C2F9695969529
:1029500080E2989FE0011124C22BD32BCE019C680A
:1029600037C08370992721E030E002C0220F331F67
:102970008A95E2F79C2F9695969540E2949FE00108
:102980001124C22BD32BCE019A6822C0D82FCC277A
:10299000CE01846F906A1CC0DC2FCC27CE01806FE3
:1029A000906A16C08C2F8F700E94971594E0D69570
:1029B000C7959A95E1F7CF70D0E0DC2FCC27D0698E
:1029C0009E01282BC90104C080E090E001C0CE0127
:1029D000DF91CF91089526E4829FC0011124FC016C
:1029E00027E0729FE00DF11D1124E60FF11DEE0F9F
:1029F000FF1FEA5AFE4F8591949108950E94EB14AF
:102A00000E94D91308958238910569F1B0F4813399
:102A1000910509F46DC048F48932910509F463C049
:102A20008A32910509F469C008958533910509F446
:102A300055C089339105B9F00895833E910569F138
:102A400038F4803E9105B1F0823E910509F1089578
:102A5000863E9105A9F1873E9105B9F1843E910525
:102A600009F064C023C02091690320FD4FC021FDFF
:102A70004DC008958091690380FD44C080916A0330
:102A800080FF44C08091690384FD42C083EE4DC045
:102A90008091690382FF38C0F5CF8091690382FD80
:102AA00033C080916A0380FD31C0ECCF80916A030E
:102AB00081FF32C08091690384FD2AC087EE35C052
:102AC0008091690383FF26C0F5CF8091690383FD60
:102AD00021C080916A0381FD1FC0ECCF8091690302
:102AE00085FD1CC01DC08091690385FD19C016C0FD
:102AF0008091690386FD16C017C08091690386FD29
:102B000013C010C089E311C082EE0FC080EE0DC06B
:102B100080E00BC086EE09C084EE07C089E205C0E4
:102B200085E303C08AE201C081E390E008959091BB
:102B3000690392FF0DC0282F2871283019F4877F70
:102B4000846006C0282F2471243011F48B7F8860A4
:102B500093FF0DC0282F2871283119F4877E8461D6
:102B600006C0282F2471243111F48B7E88612091B6
:102B70006A0320FF0DC0382F3871383019F4877F71
:102B8000816006C0382F3171313011F48E7F88603A
:102B900021FF0DC0282F2871283119F4877E81610B
:102BA00006C0282F2171213111F48E7E886194FD99
:102BB000877E089510926503109266031092670352
:102BC000109268030895CF92DF92EF92FF926B010B
:102BD0007C010E948C1881110EC00E947027C61AB9
:102BE000D70AE80AF90AC0926503D0926603E09218
:102BF0006703F0926803FF90EF90DF90CF90089505
:102C00000F931F930E948C18882321F01F910F911E
:102C10000C9470270E947027009165031091660341
:102C20002091670330916803600F711F821F931F0B
:102C30001F910F91089508950E944712811102C0BB
:102C40000E94EF120E9452128093F9020E945A12BF
:102C500090936A03809369030E941B160E94561288
:102C6000682F70E080E090E00E94550C6091630254
:102C70007091640280916502909166020C948D0CB3
:102C8000E82FF0E0EA58FC4F80810895CF92DF9260
:102C9000EF92FF920F931F93CF93DF9387EC92E015
:102CA0000E947E0686E7E82E83E0F82EC0E0D0E0A2
:102CB00092ECC92E92E0D92E0AEB12E0DF93CF936B
:102CC000DF92CF920E9417078FEB92E00E947E0660
:102CD000F70181917F010E94FF071F928F931F933D
:102CE0000F930E94170788EB92E00E947E062196C0
:102CF0008DB79EB708960FB6F8949EBF0FBE8DBFD6
:102D0000CA30D105D9F6DF91CF911F910F91FF9075
:102D1000EF90DF90CF90089580EA8A95F1F70895BB
:102D200000C008950C948C1608950C9494160C947D
:102D300095160C9494160C9499160C949416FF9274
:102D40000F931F93CF93DF9300D000D01F92CDB786
:102D5000DEB70E948C18609180038823E9F185E03A
:102D6000F82E8E010F5F1F4FF8018F2D11928A955B
:102D7000E9F7862F90E0B8018A589C4F0E94BC1852
:102D8000882389F080916B0390E045E050E0B80122
:102D90008A589C4F0E94DB2F21E02093FA02892B56
:102DA00061F410E016C08091FA028823D1F3F80193
:102DB0001192FA94E9F71092FA02A0916B03B0E035
:102DC000AA58BC4F85E0F80101900D928A95E1F771
:102DD00011E00E9474070DC070E06A587C4F80912A
:102DE0006B0390E08A589C4F0E9458190E949D16D0
:102DF00010E0812F0F900F900F900F900F90DF91A8
:102E0000CF911F910F91FF900895F894E82FE295CC
:102E1000EF70F0E031A1282F2F7081E090E001C029
:102E2000880F2A95EAF7982F9095932391A392A162
:102E3000892B82A3789408950F931F93CF93DF93E8
:102E4000CBE0D1E089918F3F11F00E94051781E01E
:102E5000C031D807B9F7C4E0D1E00BE011E08991A7
:102E60008F3F11F00E9405170C171D07C1F7DF9166
:102E7000CF911F910F910895CF92DF92EF92FF9221
:102E80000F931F93CF93DF938C01C62FD0E0CE0119
:102E9000855F9E4F7C01FC0190819F3F09F447C0F4
:102EA000D62EF894E92FE295EF70F0E081A19F70A3
:102EB00021E030E001C0220F9A95EAF7822B81A32E
:102EC00082A12095282322A378940E949016E4E002
:102ED000F1E04BE051E031E0C12C21912F3F89F02E
:102EE000A22FA295AF70B0E090968C9190E02F70D9
:102EF00002C0959587952A95E2F780FD02C0832F41
:102F000001C080E0C82A330F4E175F0731F7F70181
:102F100080818F3F11F00E94051761E0C11001C050
:102F200060E08D2D0E949216C00FD11FC882DF91E4
:102F3000CF911F910F91FF90EF90DF90CF90089568
:102F4000CF93DF93CDB7DEB72C970FB6F894DEBFE3
:102F50000FBECDBF80911001811127C085E0EEE347
:102F6000F1E0DE01189601900D928A95E1F7FE01DD
:102F70003896ABE0B1E0CE010D969F0141914D93A3
:102F8000E817F907D9F787E0E3E4F1E0DE011196ED
:102F900001900D928A95E1F7FE013196A4E0B1E02F
:102FA00081918D93E217F307D9F780911001811178
:102FB00002C095E001C090E09093800385E0891BFA
:102FC00080936B030E941C178AE0E6E7F3E0DF01C1
:102FD000982F1D929A95E9F7ECE6F3E0DF011D9238
:102FE0008A95E9F785E00E9453182C960FB6F8945D
:102FF000DEBF0FBECDBFDF91CF910C947207EF9271
:10300000FF920F931F93CF93DF93CDB7DEB72A972D
:103010000FB6F894DEBF0FBECDBF8E010F5F1F4FFE
:103020008AE0F80111928A95E9F7F12C6F2DC80119
:103030000E943C17F394F5E0FF12F8CF4AE050E00D
:10304000B8018CE693E00E94DB2F7C0121E0892B04
:1030500009F420E0E114F10441F08AE0F801ACE663
:10306000B3E001900D928A95E1F76091800370E0E2
:103070006A587C4F45E08CE693E00E945418EF2894
:1030800019F40E949F1602C081E090E02A960FB6C4
:10309000F894DEBF0FBECDBFDF91CF911F910F918E
:1030A000FF90EF9008950895FF920F931F93CF9391
:1030B000DF938C01F62ED72FC42F222349F081E015
:1030C0008093FD020E9464279093FC028093FB0290
:1030D0008091FD028823C1F08091FB029091FC0257
:1030E0000E947C27029780F0EF2DFD2FD8014C2FF6
:1030F00050E0CD01801B910B841795071CF48D9136
:103100008193F7CF1092FD02DF91CF911F910F9124
:10311000FF9008950C94F1128091000381110DC06D
:103120000E94942F811102C082E001C081E080934F
:103130000003823011F40E948F2F81E090910003F0
:10314000913009F080E008950E948A188093100160
:103150000E948C1881110C94061908950E948C18F5
:10316000811102C00C940819089581E09091010327
:103170009A3008F080E00895EF92FF920F931F932A
:10318000CF938C017B01C0910103CA3038F4B701A1
:10319000C8010E945619811126C00AC08091FE0202
:1031A0009091FF020E947C27843F914080F719C0D4
:1031B000809101038F3F19F08F5F8093010380910D
:1031C00001038A30E0F00E9464279093FF0280930D
:1031D000FE028091F90280FF04C089EE92E00E9415
:1031E0007E0680E00DC0CA3040F08091F90280FF79
:1031F00004C086ED92E00E947E061092010381E0F9
:10320000CF911F910F91FF90EF9008950C94D623CA
:103210000C94D923DF92EF92FF920F931F93CF93D9
:10322000DF937901C82F880FDD0B41155105A9F0F7
:10323000FE0193E0EE0FFF1F9A95E1F7EF5EFE4F60
:10324000818192818E5F9C4F208130E0421753072D
:1032500008F49A01A9010E94E82FCE010E94C2241D
:10326000D82E8823D1F001151105B9F083E0CC0FD9
:10327000DD1F8A95E1F7FE01EF5EFE4F438150E0CE
:103280000417150708F4A801CF5EDE4F6C817D811D
:103290006E5F7C4FC7010E94E82F8D2DDF91CF918B
:1032A0001F910F91FF90EF90DF9008950C948C1A6E
:1032B0000C94AC1A0F931F93CF93DF9300D000D0E0
:1032C000CDB7DEB76091190370911A0380911B038B
:1032D00090911C030E948B2764367105810591052E
:1032E00028F10E940016DC01CB010296A11DB11D40
:1032F00089839A83AB83BC8300E010E020E030E058
:1033000044E050E0BE016F5F7F4F82E00E940A19E7
:10331000182F882361F00E9470276093190370931F
:103320001A0380931B0390931C0301C011E0812FAB
:103330000F900F900F900F90DF91CF911F910F91F1
:1033400008958F929F92AF92BF92CF92DF92EF92A9
:10335000FF920F931F93CF93DF937C015B01942E19
:10336000852E69010E94B518811103C001E010E0AB
:1033700002C00AE010E0C1E0D0E0F894B501C70156
:10338000F60109957894811129C021960C171D0723
:103390008CF0CC9F9001CD9F300D300D112480E03A
:1033A00090E045E34A95F1F70000019628173907A8
:1033B000C1F7E3CF9091F902892F817090FF0FC080
:1033C0008F929F928FE193E09F938F930E941707B4
:1033D0000F900F900F900F9080E001C081E0DF917F
:1033E000CF911F910F91FF90EF90DF90CF90BF9002
:1033F000AF909F908F900895AF92BF92CF92DF923F
:10340000EF92FF920F931F93CF93DF9300D000D0E2
:1034100000D0CDB7DEB77B01C090AC01D090AD013C
:1034200001E010E09E012A5F3F4F40E050E060E085
:1034300070E080E00E940A19182F882309F43EC02A
:1034400056018FEFA81AB80A609115037091160300
:1034500080911703909118030E948B2764367105A1
:103460008105910518F105E010E09E012F5F3F4FA7
:1034700040E050E060E070E081E00E940A19182FFF
:1034800065E070E0C5010E940B1E91E02E812813BB
:1034900090E0192339F10E9470276093150370930F
:1034A0001603809317039093180311C065E070E032
:1034B000C5010E940B1E9E818913D5CF85E0F601C0
:1034C0003196DE01119601900D928A95E1F7112354
:1034D00049F085E0FE013196A0E1B3E001900D9244
:1034E0008A95E1F785E0E0E1F3E0D70101900D92E4
:1034F0008A95E1F7812F26960FB6F894DEBF0FBEAE
:10350000CDBFDF91CF911F910F91FF90EF90DF9092
:10351000CF90BF90AF9008950F931F93CF93DF93F9
:10352000EC018B012CEF39E14EEA51E00E94A11928
:10353000882361F02AE539E14BEB51E0B801CE0177
:10354000DF91CF911F910F910C94A11980E0DF9131
:10355000CF911F910F9108950F931F93CF93DF93F6
:10356000F894C091AC01D091AD01CE01019625E057
:10357000FB01DC0101900D922A95E1F765E070E016
:103580000E940B1E88837894F8946E817F818885D1
:10359000998500910C0310910D0320910E03309139
:1035A0000F03601771078207930751F060930C03B4
:1035B00070930D0380930E0390930F030E94E31505
:1035C0007894DF91CF911F910F9108950E94552A11
:1035D0000E943B130C94612A0E94652A0E94D11319
:1035E0000C94832A0E9402270E943C2A0E942913DD
:1035F0000E94E61A0E94EC1A0E943313FBCF8091BE
:10360000230380FF06C060912E0170E0660F771FD4
:1036100026C081FF04C060912E0184E005C082FFB6
:1036200007C060912E0188E0689FB001112417C087
:10363000909122039923D1F060912D01961788F77C
:1036400020912E0188E0289F90011124929FA001D3
:10365000939F500D112470E0CA010E94AD2F603875
:10366000710540F46115710519F406C068E070E059
:10367000862F08958FE7089581E0089580912303B0
:1036800080FF08C060912A0170E075956795759577
:10369000679521C081FF06C060912A0170E0759591
:1036A000679519C082FF04C060912A0170E010C0C4
:1036B00090912103992399F0609129019617A0F721
:1036C00080912A01899FC001112470E00E94AD2FD2
:1036D0006038710540F46115710519F406C061E0A8
:1036E00070E0862F08958FE7089581E008958D3E5C
:1036F00021F40E94FF1A819504C08E3E29F40E9495
:10370000FF1A8093270308958F3E21F40E94FF1A29
:10371000819504C0803F29F40E94FF1A80932603FC
:103720000895893F19F40E943E1B05C08A3F31F479
:103730000E943E1B81958093280308958B3F21F4BE
:103740000E943E1B819504C08C3F29F40E943E1BC1
:103750008093290308959FE0980F983078F421E032
:1037600030E0A90102C0440F551F9A95E2F7CA0143
:1037700090912503892B8093250308958D3F21F493
:103780008091230381600BC08E3F21F4809123033D
:10379000826005C08F3F29F4809123038460809369
:1037A000230308958D3E39F49091270397FF35C088
:1037B0001092270359C08E3E29F4909127031916C1
:1037C000BCF32BC0909126038F3E29F497FF25C0B0
:1037D0001092260349C0803F19F41916CCF31DC07E
:1037E00090912803893F29F41916BCF410922803FC
:1037F0003BC08A3F19F497FF10C0F8CF8B3F39F4D4
:103800009091290397FF09C0109229032DC08C3F86
:1038100021F4909129031916BCF39FE0980F98307A
:1038200080F421E030E0A90102C0440F551F9A95B1
:10383000E2F7CA018095909125038923809325039F
:1038400013C08D3F21F4809123038E7F0BC08E3FE8
:1038500021F4809123038D7F05C08F3F29F480914F
:1038600023038B7F8093230380912603811106C05D
:1038700080912703811102C01092220380912803B6
:10388000811106C080912903811102C01092210389
:1038900008958091F90283FF7EC08CE593E00E9439
:1038A0007E06809125031F928F9387E593E09F9377
:1038B0008F930E94170785E593E00E947E06809112
:1038C0002603282F082E000C330B3F938F9382E59D
:1038D00093E09F938F930E94170780E593E00E94E7
:1038E0007E0680912703282F082E000C330B3F9370
:1038F0008F938DE493E09F938F930E9417078BE43F
:1039000093E00E947E0680912803282F082E000C49
:10391000330B3F938F9388E493E09F938F930E94A0
:10392000170786E493E00E947E0680912903282FE2
:10393000082E000C330B3F938F9383E493E09F9307
:103940008F930E94170780E493E00E947E06809187
:1039500022031F928F938DE393E09F938F930E9496
:1039600017078BE393E00E947E06809123031F924A
:103970008F9388E393E09F938F930E94170785E3CB
:1039800093E00E947E068DB79EB74C960FB6F894D2
:103990009EBF0FBE8DBF0E94642720912603211178
:1039A00004C020912703222321F0909320038093C9
:1039B0001F0320912803211104C0209129032223F1
:1039C00021F090931E0380931D0384E293E00C94F6
:1039D000AF25EF92FF920F931F93CF93DF9300D009
:1039E00000D000D0CDB7DEB786E0E4E2F3E0DE0140
:1039F000119601900D928A95E1F7E0902603F090E0
:103A00002703009128031091290310922603109296
:103A100027031092280310922903E11003C0FF200E
:103A200009F45DC080911F03909120030E947C27C0
:103A3000AC0190912203992339F020912F0130E0BD
:103A40002417350758F04BC0209130018AE0289F99
:103A5000900111242417350718F041C09F3F19F039
:103A60009F5F90932203EE2061F00E94FF1A1E14C4
:103A700014F09FEF01C091E0989F902D1124909336
:103A80002603FF2061F00E94FF1A1F1414F09FEF1D
:103A900001C091E0989F902D1124909327033091BD
:103AA00026033323E1F0209127032223C1F045EBC5
:103AB0003403C0011124992319F09093260303C005
:103AC00081E08093260335EB2303C0011124992361
:103AD00019F09093270303C081E08093270301111D
:103AE00003C0112309F45DC080911D0390911E0352
:103AF0000E947C27AC0190912103992339F02091F9
:103B00002B0130E02417350758F04BC020912C01D1
:103B10008AE0289F900111242417350718F041C02E
:103B20009F3F19F09F5F90932103002361F00E9453
:103B30003E1B101614F09FEF01C091E0989F902D4E
:103B4000112490932803112361F00E943E1B11164B
:103B500014F09FEF01C091E0989F902D1124909355
:103B60002903309128033323E1F0209129032223F4
:103B7000C1F045EB3403C0011124992319F090934F
:103B8000280303C081E08093280335EB2303C001A1
:103B90001124992319F09093290303C081E08093A5
:103BA00029038091260381110BC080912703811185
:103BB00007C080912803811103C0809129038111DE
:103BC0000E94491CEB82FC820D831E8386E0FE016D
:103BD0003196A4E2B3E001900D928A95E1F7269622
:103BE0000FB6F894DEBF0FBECDBFDF91CF911F910E
:103BF0000F91FF90EF900895E4E2F3E086E0DF019B
:103C00001D928A95E9F710922203109221031092D7
:103C1000230308950895FC01680F791F8FEF91E346
:103C2000E617F70771F02191822728E030E087FF3F
:103C300003C0880F892701C0880F21503109B9F7C7
:103C4000EFCF0895CF93DF93EC01FB0182818823AE
:103C500009F43CC1C430FDE5DF0760F4CB3F9CE5CF
:103C6000D90788F49E0122503C452431310508F0E3
:103C70002EC109C0C236EDE5DE0729F0C63AFDE5E2
:103C8000DF0709F024C10E945A1290936A038093BF
:103C90006903C1318CE5D80709F4C6C008F042C0F9
:103CA000C930ECE5DE0709F49BC000F5C5308CE5B2
:103CB000D80709F485C078F4C330ECE5DE0709F4D1
:103CC00078C008F07AC0C230DC4509F0F5C08091B8
:103CD00069038160EFC0C7309CE5D90709F478C05B
:103CE00008F07AC0809169038061E4C0CD30FCE5C2
:103CF000DF0709F487C058F4CB309CE5D90709F4F5
:103D000079C008F07BC08091690388606FC0CF30B4
:103D1000FCE5DF0709F480C008F082C080916903E8
:103D2000877FC8C0CE3F9CE5D90709F471C000F574
:103D3000C531FCE5DF0709F485C068F4C3319CE5B3
:103D4000D90709F475C008F095C00E94FD0B809159
:103D500069038F77AFC0CC3FFCE5DF07A9F108F01E
:103D600054C0CB3FDC4509F0A7C080916A0340C036
:103D7000C230EDE5DE0709F489C058F4C1158DE5C0
:103D8000D80709F45AC008F069C080916A038260BC
:103D90002FC0C236EDE5DE0709F47CC0C63AFDE56A
:103DA000DF0709F481C0C330DD4509F085C080E03C
:103DB0006EC08091690382607DC08091690316C0E6
:103DC00080916903886076C080916A0382604FC0E9
:103DD0008091690380626EC08091690380646AC0CB
:103DE0000E94FD0B80916903806864C0846062C09A
:103DF00081603DC0809169038E7F5CC080916903C2
:103E00008D7F58C08091690316C080916A0318C0E5
:103E100080916A038D7F2BC0809169038F7E4AC099
:103E2000809169038F7D46C0809169038F7B42C07A
:103E300080916903877F8B7F3DC080916A038D7F6E
:103E40008E7F15C08091690382FB222720F991E0C3
:103E5000922790FB82F990FB83F92CC080916A0332
:103E6000982F909591708E7F892B90FB81F980938C
:103E70006A0322C00E94FD0B8091690387FB222701
:103E800020F991E0922790FB87F914C081E00E940D
:103E9000FB1212C08091690384FB222720F991E074
:103EA000922790FB84F906C080916903982F909522
:103EB00090FB80F9809369038091690390916A0374
:103EC0000E946B120E94FD0B80E001C081E0DF9137
:103ED000CF910895809129011F928F9380912A019B
:103EE0001F928F9380912D011F928F9380912E01AD
:103EF0001F928F9380912F011F928F938091300199
:103F00001F928F938FE793E09F938F930E941707E1
:103F10008DB79EB70E960FB6F8949EBF0FBE8DBF9D
:103F20000895883220F58E3108F068C08B3091F109
:103F3000C0F4873009F0BEC081E08093300184E195
:103F400080932F018AE080932E018EE180932D01D2
:103F500088E080932A0188E28093290181EE94E031
:103F6000C6C0833109F443C0843169F1A3C08F34E2
:103F700009F49EC028F4893231F1883359F09AC08F
:103F8000813531F008F4D4C0823509F4A7C092C05D
:103F90008FEFA5C083E095E00E947E060E946A1F15
:103FA0001F9281E08F931F9288E08F938CEF93E0B4
:103FB0009F938F930E9417070F900F900F900F9071
:103FC0000F900F9096C080E095E00E947E06809151
:103FD0002E03882309F4AAC010922E0310922D03F9
:103FE00010922C0310922B0310922A03B1C082EF7F
:103FF00094E00E947E060E946A1F7BC08D518093D0
:104000002E03833031F170F48130D1F0823009F029
:104010003FC08FE291E090932D0380932C0383EDBA
:1040200091E01FC0853059F108F1863089F589E2A9
:1040300091E090932D0380932C038EE092E011C0C9
:1040400080E391E090932D0380932C038AEC91E020
:1040500008C08EE291E090932D0380932C038FEDA6
:1040600091E090932B0380932A0318C08DE291E096
:1040700090932D0380932C038CEE91E0F2CF8AE293
:1040800091E090932D0380932C038BEF91E0E9CF87
:1040900010922E038FEE94E00E947E0680912E03F4
:1040A000882309F455C01F928F938BEE94E00DC0C6
:1040B0008AE015C08EED94E01AC097FF47C01082C9
:1040C00080811F928F9388ED94E09F938F930E943D
:1040D00017070F900F900F900F900BC081E0E091A9
:1040E0002C03F0912D03309729F585ED94E00E9483
:1040F0007E0620912E03222359F180912A0390916C
:104100002B03009711F486EC91E09F938F931F92FD
:104110002F938CEC94E09F938F930E9417070F903E
:104120000F900F900F900F900F9016C080E00895A1
:1041300086EFD5CF2081082E000C990B820F911DA0
:104140008F3F910509F00CF4B8CF8FEF8083B8CF83
:1041500088EC94E00E947E0681E00895CF93C82FFA
:104160001F928F9389E195E09F938F930E94170789
:1041700081E090E0A0E0B0E0BC01CD0104C0660F9A
:10418000771F881F991FCA95D2F70E94550C0F9070
:104190000F900F900F90CF910C94FD0BDF92EF9248
:1041A000FF920F931F93CF93DF93482F50E0FA01B4
:1041B0003597EF33F10508F03FC1EE59FF4F0C94EE
:1041C000C12F0E9456121F928F9381E799E09F930F
:1041D0008F930E9417070E94521283FB992790F930
:1041E0001F929F9382FB992790F91F929F9381FBC7
:1041F000992790F91F929F93982F91701F929F93E8
:104200001F928F9388E299E09F938F930E941707E4
:104210000E945A1287FB222720F91F922F9386FBB8
:10422000222720F91F922F9385FB222720F91F9226
:104230002F9384FB222720F91F922F9383FB2227A1
:1042400020F91F922F9382FB222720F91F922F9390
:1042500091FB222720F91F922F93292F21701F9263
:104260002F9381FB222720F91F922F93282F217053
:104270001F922F939F938F9383E498E09F938F9344
:104280000E9417078DB79EB788960FB6F8949EBF09
:104290000FBE8DBF06C081E39AE00E947E060E9499
:1042A000EF12C1E0CEC081E996E074C08091F902BE
:1042B000817F8E7F8093F9028AE696E00E947E06D7
:1042C0008DE29AE00E947E0681E080932F03E9CF81
:1042D00081E19AE00E947E060E947707E2CF8091FA
:1042E000F902C82FC095C170C0FB80F98093F90214
:1042F000CC2319F085E09AE091C088EF99E00E9404
:104300007E068091F902897F877F8093F902C9CF69
:104310009091F90291FBCC27C0F981E0C827892F41
:10432000C0FB81F98093F902CC2319F08BEE99E060
:1043300027C08DED99E02EC09091F90292FBCC2719
:10434000C0F981E0C827892FC0FB82F98093F90268
:10435000CC2319F08EEC99E013C08EEB99E01AC0D3
:104360009091F90293FBCC27C0F981E0C827892FEF
:10437000C0FB83F98093F902CC2351F082EB99E0E2
:104380000E947E068091F90281608093F90259C0F3
:1043900085EA99E00E947E0684CF82EA95E0FACF12
:1043A0000E947027062FF72EE82ED92EC0916903A0
:1043B000C7FBCC27C0F910916403D0913D010E9446
:1043C0004725DF92EF92FF920F931F92CF931F9298
:1043D0001F931F92DF931F928F938EE195E09F931F
:1043E0008F930E9417078DB79EB70E960FB6F8945D
:1043F0009EBF0FBE8DBF55CF0E94FD0B90916903EC
:1044000097FBCC27C0F981E0C827892FC0FB87F92B
:1044100080936903CC2329F08BE999E00E947E0602
:1044200010C080E999E0B6CF895303C08D5101C017
:1044300080E00E94AE2035CF8EE899E00E947E0693
:10444000C0E08C2FDF91CF911F910F91FF90EF90E3
:10445000DF90089580E008950C942A22CF93C82F0E
:1044600080912F03813071F040F0823009F045C017
:104470008C2F0E94911F81E046C00E945011823211
:10448000F1F504C00E945011823261F48C2F0E9419
:104490002C22811104C08C2F0E94CE202CC081E0E0
:1044A00090E029C08C2F0E942A22811123C0C431A0
:1044B000C9F058F4CB3069F0C031B9F482E0809390
:1044C0002F0388E30E94911F15C0C93259F0C833E9
:1044D00061F48AE696E00E947E0685E195E00E94FE
:1044E0007E0608C010922F030CC083E195E00E9465
:1044F0007E0607C081E0817006C010922F0380E025
:1045000002C080E0F8CFCF910895CF93DF9386313A
:104510009C4541F5EB010E945011982F8A81209112
:10452000020130910301882379F09A7A81E009F43D
:1045300080E080933003911102C069E201C065E31D
:10454000C9010E94A1260AC080913003811102C0D6
:1045500069E201C065E3C9010E94AC260E94921184
:1045600080E001C081E0DF91CF9108950F931F9308
:10457000CF93DF93C42FD22FFC0182818823C9F00F
:10458000409333030E946427909332038093310356
:1045900080E28C0F883008F057C0C77081E001C0FE
:1045A000880FCA95EAF7DF91CF911F910F910C9474
:1045B0005A0980913303481330C0809131039091A0
:1045C00032030E947C27883C910538F510E21D0FCC
:1045D000CD17B9F080E28C0F883040F4C77081E0CD
:1045E00001C0880FCA95EAF70E946109183028F5C2
:1045F00081E09D2F977001C0880F9A95EAF70E947D
:104600005A09802F0E9451091830F0F4D77081E0C8
:1046100001C0880FDA95EAF70AC080E28C0F883073
:1046200098F4C77081E001C0880FCA95EAF7DF915E
:10463000CF911F910F910C946109802FDF91CF9141
:104640001F910F910C945109DF91CF911F910F9100
:1046500008950F939C01CB01243F4CE5340731F1C1
:1046600088F4293DFCE53F07D9F02A3D4CE53407A5
:1046700079F1283D3C45A9F506E221EE41EE68EDD1
:104680007CE52BC0263FFCE53F07E1F0A8F0273F83
:104690003C4539F507E225EE46EE67EF7CE51DC0A7
:1046A00007E225EE45EE69ED7CE517C006E221EE56
:1046B00040EE64EF7CE511C007E225EE44EE65EFC5
:1046C0007CE50BC006E221EE42EE66EF7CE505C01C
:1046D00008E221E045EE6AED7CE50E94B62280E02A
:1046E00008C0FC018281882319F01092330301C0B5
:1046F00081E00F9108958EE1489B02C08150E1F75F
:10470000489BFECF0895589880E28A95F1F7589A11
:104710000895FC012AE02A95F1F728E090E080E076
:1047200031E040E14A95F1F7880F489B02C0816073
:10473000932700C0000040E14A95F1F7215089F726
:1047400020E12A95F1F729B100C0000030E13A9547
:10475000F1F7217092272081920F90830895EF92B4
:10476000FF920F931F93CF93DF931F92CDB7DEB7C6
:1047700019828C017C01E60EF11C0E151F0551F00B
:104780000E947B23CE0101960E948923F801819328
:104790008F01F3CF81E09981911180E00F90DF913B
:1047A000CF911F910F91FF90EF900895509A589AD2
:1047B00008955098589AE89AE9E6F0E080818C7F55
:1047C00080830895615091E001C0990F6A95EAF7DE
:1047D00020E031E0992361F0492F482319F0589ADD
:1047E000232701C0589840E24A95F1F79695F2CFF9
:1047F000222311F0589A01C0589880E28A95F1F767
:1048000058980895FF920F931F93CF93DF93EC0175
:104810008C01060F111DC017D10741F0F9900E94BD
:10482000832368E08F2D0E94E223F5CFDF91CF91A3
:104830001F910F91FF9008951F920F920FB60F9244
:1048400011240F931F932F933F934F935F936F9375
:104850007F938F939F93AF93BF93EF93FF93CF93E8
:10486000DF931F92CDB7DEB719820E947B23CE0162
:1048700001960E948923082F069506950695902F8C
:1048800096959570202F2570920F292F237096955D
:104890009695920F877089135FC0898181115CC0E2
:1048A000043008F059C080E18A95F1F7589A509A7F
:1048B00082E08A95F1F700C0589888E0089F80014F
:1048C0001124D801AF5EBE4F1696ED91FC9117975B
:1048D0003097A9F06091AC017091AD0114962D91C3
:1048E0003C911597260F371F11968D919C91129729
:1048F000680F791F13964C9113978C910995F801C5
:10490000EF5EFE4F6381662351F08091AC01909180
:10491000AD0124813581820F931F0E9402240E94E1
:10492000832380E18A95F1F758985098589A80E14E
:104930008A95F1F7F801EF5EFE4F6081662351F032
:104940008091AC019091AD0121813281820F931F42
:104950000E94AF230E947B230F90DF91CF91FF91A4
:10496000EF91BF91AF919F918F917F916F915F91E7
:104970004F913F912F911F910F910F900FBE0F906C
:104980001F9018950F931F93CF93DF938430910559
:104990000CF06DC0EC01F894509A589885E08A9517
:1049A000F1F700009C2F969595702C2F2570920F93
:1049B000892F83709695969523E0CC0FDD1F2A955D
:1049C000E1F7980F8E01092B0E94832384E08A95DA
:1049D000F1F700C068E0802F0E94E22380E18A9511
:1049E000F1F75098589A489902C000C0FCCF87E070
:1049F00090E0489B08C0019721F4509A589A789407
:104A000036C000C0F6CFFE01EF5EFE4F6381662325
:104A100081F08091AC019091AD0124813581820FAC
:104A2000931F0E94AF23811104C0509A589A789422
:104A30001FC00E947B2380E28A95F1F75898509A14
:104A400080E18A95F1F7CF5EDE4F6881662351F0F1
:104A50008091AC019091AD0129813A81820F931F21
:104A60000E9402240E948323789481E001C080E0A8
:104A7000DF91CF911F910F9108959093330280930E
:104A80003202089590933A038093390308950E9467
:104A90008C18811103C0809134030895E09139038B
:104AA000F0913A03309721F00190F081E02D0994C4
:104AB00080E00895EF92FF921F93CF93DF93FC0164
:104AC000A0913903B0913A03109709F442C0809144
:104AD0003D01882341F08091690387FF04C08081F4
:104AE000818386E08083EF011296ED91FC9113970C
:104AF000CE0109958091F90282FF2BC080FF04C08E
:104B00008AE49AE00E947E0618E084E4E82E8AE0B7
:104B1000F82E8091F90280FF0BC088811F928F933D
:104B2000FF92EF920E9417070F900F900F900F9037
:104B3000115021961111EDCF8091F90280FF09C02B
:104B400082E49AE0DF91CF911F91FF90EF900C9457
:104B50007E06DF91CF911F91FF90EF900895E09135
:104B60003903F0913A03309739F022E0DC012C93BD
:104B70000480F581E02D0994089520913703309148
:104B800038032817390771F090933803809337035F
:104B9000E0913903F0913A03309721F00680F781D4
:104BA000E02D09940895209135033091360328179C
:104BB000390771F09093360380933503E091390300
:104BC000F0913A03309721F00084F185E02D0994AB
:104BD0000895FC01329680913D01882331F0809147
:104BE000690387FF02C09EE101C096E080E091501A
:104BF00028F021912223D9F38F5FF9CF08956623FE
:104C000051F120913D012223E9F02091690327FF12
:104C100019C0462F4695469546954E31E0F467708B
:104C200021E030E002C0220F331F6A95E2F7FC0159
:104C3000E40FF11D828190E02823392381E0232BAA
:104C400069F409C0FC01329608962191621729F097
:104C5000E817F907D1F780E0089581E008959C01F5
:104C6000FC0132969FEF80E04191461789F09F3F0B
:104C700019F4411101C0982F8F5F8630A9F79F3F2B
:104C800039F0F901E90FF11D97FDFA956283089556
:104C900008959C012A5F3F4FFC014281461301C0E9
:104CA0001282019682179307B9F70895262F269549
:104CB000269526952E3170F4FC01E20FF11D6770E8
:104CC00021E030E001C0220F6A95EAF78281282BAB
:104CD000228308958091F90280FF0CC01F926F9388
:104CE0008AE79AE09F938F930E9417070F900F9087
:104CF0000F900F900895262F2695269526952E31F4
:104D000078F4FC01E20FF11D677021E030E001C092
:104D1000220F6A95EAF7209582812823228308953D
:104D20008091F90280FF0CC01F926F938CE59AE08E
:104D30009F938F930E9417070F900F900F900F90E3
:104D4000089520913D01222329F02091690327FD38
:104D50000C9456260C942F2620913D01222329F0F5
:104D60002091690327FD0C947B260C944926209101
:104D70003D01FC013296222331F08091690387FFC7
:104D800002C08EE101C086E0DF011D928A95E9F73D
:104D9000089508950C94C92683E080933B030C94F6
:104DA000CA26811102C081E001C082E080933B03EA
:104DB0000C94CA260C94D12681E080933B030C947A
:104DC000CA260C94DC2608950C94E3260C94E42661
:104DD0000C94E3260C94E3260C94E326CF930E94D4
:104DE000EA260E94FF170E94E826C0E08C2F0E944E
:104DF0004016811104C0CF5FCA30C1F701C081E005
:104E0000CF91089508951F920F920FB60F9211241B
:104E10008F939F93AF93BF9380913C03811113C0F5
:104E20008091810390918203A0918303B0918403C8
:104E30004196A11DB11D8093810390938203A0939D
:104E40008303B0938403BF91AF919F918F910F9093
:104E50000FBE0F901F90189580918903843031F117
:104E60000E94F70710923C0320E488E190E00FB61F
:104E7000F894A895809360000FBE2093600083B7DC
:104E8000817F846083BF83B7816083BF7894889576
:104E900083B78E7F83BF0FB6F894A895809160008A
:104EA000886180936000109260000FBE08950E9498
:104EB000FD0B0C94FB0782E084BD93E095BD9AEF57
:104EC00097BD80936E0008952FB7F8948091810369
:104ED00090918203A0918303B09184032FBF089522
:104EE0002FB7F894609181037091820380918303BE
:104EF000909184032FBF08959C014FB7F89480913F
:104F0000810390918203A0918303B09184034FBFEA
:104F1000821B930B0895CF92DF92EF92FF922FB7EF
:104F2000F894C0908103D0908203E0908303F090C6
:104F300084032FBFA7019601261B370B480B590B83
:104F4000CA01B901FF90EF90DF90CF900895789457
:104F50001F920F920FB60F9211248F939F93AF93CE
:104F6000BF938091810390918203A0918303B091BC
:104F700084030196A11DB11D809381039093820348
:104F8000A0938303B0938403BF91AF919F918F91BE
:104F90000F900FBE0F901F90189581E08093E00056
:104FA00080E28093D8001092C9008FE19EE40197BF
:104FB000F1F700C0000087E090EBDC0180939203E2
:104FC00090939303A0939403B09395039CE088E19E
:104FD0000FB6F894A895809360000FBE9093600080
:104FE000FFCF809163030895089522E02093E900A4
:104FF0002FEF3091E800215035FD06C035ED3A9590
:10500000F1F700002111F5CF2091E80025FF0BC03A
:1050100040E050E066E070E00E94F22A8091E800F3
:105020008E778093E8000895CF93DF9320913D0120
:10503000222339F02091690327FF03C060E222E0B8
:1050400002C068E021E02093E9002FEF3091E800F2
:10505000215035FD06C035ED3A95F1F700002111DC
:10506000F5CF2091E80025FF1DC0EC0180913D01A6
:10507000811105C040E050E068E070E003C070E0DE
:1050800040E050E0CE010E94F22A8091E8008E7745
:105090008093E80080E2FE01A3E4B3E001900D926A
:1050A0008A95E1F7DF91CF91089580933F03709344
:1050B00041036093400380918903843001F582E0CD
:1050C0008093E9008FEF9091E800815095FD06C034
:1050D00095ED9A95F1F700008111F5CF8091E800E8
:1050E00085FF0DC040E050E063E070E08FE393E0A7
:1050F0000E94F22A8091E8008E778093E80008955C
:10510000BC0184E00C945528BC0183E00C94552824
:105110008CEA9AE00E947E0680918803811109C082
:105120000E94832C0E94E02C8091E2008460809396
:10513000E200089588EA9AE00E947E0610928803B1
:10514000089584EA9AE00E947E060C94E12680EAA3
:105150009AE00E947E066091850381E0611101C0A2
:1051600080E00C94CC268CE99AE00E947E06909117
:10517000890381E0943009F080E0609185030C940C
:10518000D12620913E032F5F822F62E30E94A12F40
:10519000992319F020933E03089510923E038091C5
:1051A0004203882371F180918903843041F5809115
:1051B000E9008F702091EC00922F917020FD90E813
:1051C000892B93E09093E9009091EB0090FF14C03D
:1051D0009091EE0097FF10C09091E80095FF03C0FA
:1051E0001092F100F9CF9091E80090FF05C09091E6
:1051F000E8009E779093E8008F708093E90010920A
:105200004203089542E061EC81E00E94FC2B42E2FF
:1052100061EC82E00E94FC2B42E261EC83E00E94A0
:10522000FC2B9091890381E0943009F080E060913B
:1052300085030C94DA2680918B03833009F461C0D6
:1052400030F4813071F0823009F49AC008958A30C8
:1052500009F486C08B3009F46CC0893009F0A8C00D
:1052600020C080918A03813A09F0A2C08091E800B1
:10527000877F8093E80080918E0390918F03892B24
:1052800021F460E283E493E003C060E080E090E01A
:1052900070E00E943D2B8091E8008B778093E800BE
:1052A000089580918A03813209F082C080918E0333
:1052B00090918F03029708F07BC08091E800877F70
:1052C0008093E8008091E80082FD05C08091890309
:1052D0008111F8CF6DC02091F3008091F20090E031
:1052E000922B029731F48091F100813011F08630D9
:1052F00021F48091F100809363038091E8008B7723
:1053000053C080918A03813A09F052C080918E0384
:1053100090918F03892B09F04BC08091E800877F23
:105320008093E8008091E80080FFFCCF80913D01F0
:1053300036C080918A038132D9F580918E03909195
:105340008F03892BA9F58091E800877F8093E8007F
:105350000E94312C80918C0380933D010C94FD0BB5
:1053600080918A03813221F58091E800877F8093C4
:10537000E8000E94312C80918D038093640308958E
:1053800080918A03813AA1F48091E800877F80931D
:10539000E8008091E80080FFFCCF80916403809357
:1053A000F1008091E8008E778093E8000C94312C16
:1053B00008959FB7F894109242039FBF909189037C
:1053C000943009F057C09091E9009F703091EC0043
:1053D000232F217030FD20E8922B23E02093E90059
:1053E0002091EB0020FF43C02091EE0027FF3FC03B
:1053F00020913D03222321F02091E80025FF37C0B2
:1054000010923D0326E03091E80035FD15C0309143
:105410008903343061F53091EB0035FD28C021500F
:1054200021F481E080933D0322C0EFE9FFE0319752
:10543000F1F700C00000E7CF8093F1008091E80011
:1054400085FD0AC08091E80080FFFCCF8091E800D4
:105450008E778093E80006C08FB7F89421E0209300
:1054600042038FBF9F709093E90080E008959F7082
:105470009093E9008FEF089584B7877F84BF0FB6BC
:10548000F894A895809160008861809360001092E4
:1054900060000FBE90E080E80FB6F8948093610042
:1054A000909361000FBE0C94DC260E94832C0E9416
:1054B000E02CE2EEF0E080818460808378940C94AC
:1054C000742F81E391E00C9442258091890385300B
:1054D000C9F488E99AE00E947E06809189038530AC
:1054E00079F40E942C27809187038823B1F30E94CE
:1054F000EE26882391F30E94DC2A0E94FD0BEDCF5B
:105500000C945727089508950C94862A292F332741
:1055100023303105C9F060F42130310581F02230AB
:10552000310509F041C08BE590E02AEE3AE040C039
:1055300021323105E1F02232310531F135C082E10D
:1055400090E025E43BE034C099278130910549F093
:1055500028F0029749F5E0EBFAE005C0E6EEFAE044
:1055600002C0E2ECFAE0849190E09F0121C0633038
:105570007105D0F4660F771FFB01E45DFD4F2081BC
:10558000318189E090E014C06330710568F4FB015B
:10559000EE0FFF1FEA5DFD4F20813181FB01ED5DC4
:1055A000FD4F808190E004C080E090E020E030E09A
:1055B000FA0131832083089580E189BD82E189BDAC
:1055C00009B400FEFDCF8091D8008F7D8093D80074
:1055D0008091E00082608093E0008091E00081FD96
:1055E000FCCF0895CF92DF92EF92FF920F931F931B
:1055F000CF93DF93EC018B017A010E94502C811133
:1056000033C0E114F10439F0F70180819181081B66
:10561000190BC80FD91FC12CD12C0115110519F177
:105620008091E80085FD16C08091E8008E77809318
:10563000E800E114F10449F0F70180819181C80E7E
:10564000D91ED182C08285E00FC00E94502C8823D1
:1056500021F30AC089918093F10001501109FFEFF5
:10566000CF1ADF0ADACF80E0DF91CF911F910F913F
:10567000FF90EF90DF90CF900895209190033091AC
:1056800091032617370748F06115710539F4209109
:10569000E8002E772093E80001C0B901FC0120E06A
:1056A0006115710579F1809189038823F1F18530C5
:1056B000F1F18091E80083FD3CC08091E80082FD1B
:1056C0002EC08091E80080FFEBCF2091F300809105
:1056D000F20090E0922B6115710551F08830910530
:1056E00038F421912093F100615071090196F3CFB4
:1056F00021E0089709F020E08091E8008E77809300
:10570000E800CECF2111CFCF0AC080918903882332
:1057100061F0853061F08091E80083FD0AC08091DE
:10572000E80082FFF2CF80E0089582E0089583E0F0
:10573000089581E0089520919003309191032617F8
:10574000370748F06115710539F42091E8002E778C
:105750002093E80001C0B901FC0120E0611571054A
:1057600091F180918903882309F440C0853009F4C0
:105770003FC08091E80083FD3DC08091E80082FD3C
:105780002FC08091E80080FFE9CF2091F300809145
:10579000F20090E0922B6115710559F08830910567
:1057A00040F424912093F1003196615071090196E3
:1057B000F2CF21E0089709F020E08091E8008E7791
:1057C0008093E800CBCF2111CCCF0AC08091890310
:1057D000882361F0853061F08091E80083FD0AC084
:1057E0008091E80082FFF2CF80E0089582E0089582
:1057F00083E0089581E00895982F973068F590939D
:10580000E900981739F07091EC002091ED0050916B
:10581000F00003C0242F762F50E021FD02C09F5FCF
:10582000ECCF3091EB003E7F3093EB003091ED00F8
:105830003D7F3093ED003091EB0031603093EB0011
:105840007093EC002093ED005093F0002091EE0057
:1058500027FDE5CF80E008958F708093E90081E017
:10586000089580918A0387FF11C08091E80082FD2E
:1058700005C0809189038111F8CF11C08091E800A3
:105880008B770BC080918903882349F08091E800D1
:1058900080FFF8CF8091E8008E778093E80008952C
:1058A0002091E4003091E50095E64091EC00842FD2
:1058B000817040FF23C08091E80080FD1DC0809171
:1058C0008903882399F0853099F08091EB0085FD5C
:1058D00011C04091E4005091E5002417350729F3E9
:1058E000915011F09A01E1CF84E0089582E008958B
:1058F00083E0089581E0089580E008954091E800F4
:1059000042FFDDCF08950E94F12C0E94F92CE0EEB9
:10591000F0E0808181608083E8EDF0E080818F7726
:10592000808319BCA7EDB0E08C918E7F8C93808131
:105930008F7E80831092880308950F931F93CF93D7
:10594000DF930E94F12C0E94F92CC8EDD0E08881F1
:105950008F77888388818068888388818F7D88831A
:1059600019BC10928903109285031092870310923C
:10597000860300EE10E0F80180818B7F80838881B0
:105980008160888342E060E080E00E94FC2BE1EED1
:10599000F0E080818E7F8083E2EEF0E080818160A4
:1059A0008083808188608083F80180818E7F8083FE
:1059B000888180618883DF91CF911F910F91089535
:1059C000E8EDF0E080818F7E8083E7EDF0E080817C
:1059D0008160808384E082BF81E0809388030C949F
:1059E0009D2CE8EDF0E080818E7F80831092E200B4
:1059F00008951092DA001092E10008951F920F921C
:105A00000FB60F9211242F933F934F935F936F9391
:105A10007F938F939F93AF93BF93EF93FF93809167
:105A2000E10082FF0BC08091E20082FF07C08091FD
:105A3000E1008B7F8093E1000E94C1288091DA0011
:105A400080FF1FC08091D80080FF1BC08091DA00CA
:105A50008E7F8093DA008091D90080FF0DC080E1B5
:105A600089BD82E189BD09B400FEFDCF81E080934C
:105A700089030E94882805C019BC109289030E94DE
:105A80009A288091E10080FF19C08091E20080FF98
:105A900015C08091E2008E7F8093E2008091E20049
:105AA00080618093E2008091D80080628093D8006A
:105AB00019BC85E0809389030E94A7288091E100AA
:105AC00084FF30C08091E20084FF2CC080E189BD5A
:105AD00082E189BD09B400FEFDCF8091D8008F7DA1
:105AE0008093D8008091E1008F7E8093E1008091C7
:105AF000E2008F7E8093E2008091E20081608093DB
:105B0000E20080918503882311F084E007C0809132
:105B1000E30087FD02C081E001C083E08093890338
:105B20000E94B3288091E10083FF29C08091E200A8
:105B300083FF25C08091E100877F8093E10082E0B0
:105B400080938903109285038091E1008E7F80937A
:105B5000E1008091E2008E7F8093E2008091E2007C
:105B600080618093E20042E060E080E00E94FC2BD4
:105B70008091F00088608093F0000E94A128FF913E
:105B8000EF91BF91AF919F918F917F916F915F91B5
:105B90004F913F912F910F900FBE0F901F9018952E
:105BA0001F920F920FB60F9211242F933F934F9392
:105BB0005F936F937F938F939F93AF93BF93CF9395
:105BC000DF93EF93FF93C091E900CF708091EC00D9
:105BD000D82FD17080FDD0E81092E9008091F000BC
:105BE000877F8093F00078940E94142E1092E90031
:105BF0008091F00088608093F000CD2BCF70C0932F
:105C0000E900FF91EF91DF91CF91BF91AF919F910B
:105C10008F917F916F915F914F913F912F910F9055
:105C20000FBE0F901F9018951F93CF93DF93CDB7A2
:105C3000DEB7AA970FB6F894DEBF0FBECDBFEAE875
:105C4000F3E08091F100819323E0E239F207C9F794
:105C50000E941B298091E80083FF2EC180918A0356
:105C600090918B03492F50E04A30510508F024C130
:105C7000FA01EF55FF4F0C94C12F803821F0823884
:105C800009F01AC108C08091860390918703992377
:105C900089F082600FC080918E038F70873008F08A
:105CA0000BC18093E9008091EB0085FB882780F988
:105CB0001092E9009091E800977F9093E80080931C
:105CC000F1001092F100D1C0282F2D7F09F0F4C00F
:105CD000882319F0823061F0EFC080918C0381300D
:105CE00009F0EAC0933009F080E0809387032EC06A
:105CF00080918C0381112AC080918E038F702FEFC9
:105D0000280F263008F0D8C08093E9002091EB00DE
:105D100020FF1CC0933021F48091EB00806214C0FE
:105D20009091EB0090619093EB0021E030E0A901AD
:105D300002C0440F551F8A95E2F74093EA00109283
:105D4000EA008091EB0088608093EB001092E900FC
:105D50008091E800877F8093E8000E94312CACC0DE
:105D60008111AAC010918C031F778091E300807885
:105D7000812B8093E3008091E800877F8093E80087
:105D80000E94312C8091E80080FFFCCF8091E300DD
:105D900080688093E300111102C082E001C083E0BB
:105DA0008093890389C08058823008F085C0809133
:105DB0008C0390918D038C3D53E0950779F583E03A
:105DC0008A838AE289834FB7F894DE01139620E034
:105DD0003EE051E2E32FF0E050935700E49120FFC2
:105DE00003C0E295EF703F5FEF708E2F90E0EA30D6
:105DF00010F0C79601C0C0968D939D932F5F2431FC
:105E000049F74FBF8091E800877F8093E8006AE2FE
:105E100070E0CE0101960E943D2B16C060918E036A
:105E200070918F03AE014F5F5F4F0E94842ABC01C7
:105E3000892B09F441C09091E800977F9093E80086
:105E400089819A810E949B2B8091E8008B778093B7
:105E5000E80032C0803881F58091E800877F809328
:105E6000E800809185038093F1008091E8008E77AF
:105E700072CF811121C080918C0390918D0399275D
:105E80000297D4F48091E800877F8093E8008091A6
:105E90008C03809385030E94312C809185038111AE
:105EA00006C08091E30087FD02C081E001C084E06C
:105EB000809389030E9402298091E80083FF0AC031
:105EC0008091E800877F8093E8008091EB008062FA
:105ED0008093EB00AA960FB6F894DEBF0FBECDBF3D
:105EE000DF91CF911F910895CF93809189038823EB
:105EF000A1F0C091E900CF709091EC00892F8170E2
:105F000090FD80E8C82B1092E9008091E80083FDA5
:105F10000E94142ECF70C093E900CF9108950E9483
:105F2000832C109289030895E8EDF0E08081806170
:105F300080838AE18A95F1F700C08091D900817051
:105F40000895991B79E004C0991F961708F0961BD5
:105F5000881F7A95C9F78095089597FB072E16F448
:105F6000009407D077FD09D00E94C72F07FC05D009
:105F70003EF4909581959F4F0895709561957F4F60
:105F80000895EE0FFF1F0590F491E02D0994AA1BD0
:105F9000BB1B51E107C0AA1FBB1FA617B70710F014
:105FA000A61BB70B881F991F5A95A9F78095909546
:105FB000BC01CD010895FB01DC0104C08D9101906D
:105FC000801921F441505040C8F7881B990B08955F
:105FD000FB01DC0102C001900D9241505040D8F706
:105FE0000895F999FECF92BD81BDF89A992780B5A1
:105FF0000895A8E1B0E042E050E00C942530262F4F
:10600000F999FECF92BD81BDF89A019700B40216AE
:1060100039F01FBA20BD0FB6F894FA9AF99A0FBE5C
:1060200008950396272F0E9400300E94FF2F252FEE
:106030000E940030242F0C9400300196272F0E94DC
:1060400000300C94FF2FDC01CB01FC01F999FECF4D
:1060500006C0F2BDE1BDF89A319600B40D924150F0
:0A6060005040B8F70895F894FFCF00
:10606A00C800C50235349796F0F166F6F5F4369312
:10607A00010000000100000000000000050100000E
:10608A00000406000000000000280850011E0A143F
:10609A0001F1271428F52784288028F427019697E8
:1060AA0034F7C6313233F1F4F5F6E200E900EA00DA
:1060BA00B500B600B700CD008301CC008A01920179
:1060CA0094012102230224022502260227022A021F
:1060DA00B300B4006F007000818283E200E900EA35
:1060EA0000B500B600B700CD008301CC008A01924A
:1060FA000194012102230224022502260227022AF0
:10610A0002B300B4006F0070008182830203736CD3
:10611A006176655F6D61747269780073796E635F29
:10612A0074696D6572003F3F3F006D6B5F64656C1B
:10613A006179006D6B5F696E74657276616C006D72
:10614A006B5F6D61785F7370656564006D6B5F741A
:10615A00696D655F746F5F6D6178006D6B5F7768FD
:10616A0065656C5F6D61785F7370656564006D6B02
:10617A005F776865656C5F74696D655F746F5F6D85
:10618A0061780040B6222F0C790B570BFC0A150BCD
:02619A002E0BCA
:00000001FF
